:100000000C9438000C9453000C9453000C9453003F
:100010000C9453000C9453000C9453000C94530014
:100020000C9453000C9453000C94780C0C945300D3
:100030000C94050C0C9453000C9453000C94530036
:100040000C9453000C941D020C9453000C94140B4C
:100050000C94670B0C9453000C9453000C945300B5
:100060000C9453000C9453000C9453000C945300C4
:1000700011241FBECFEFD4E0DEBFCDBF11E0A0E062
:10008000B1E0EEEDFAE202C005900D92A038B107A2
:10009000D9F713E0A0E8B1E001C01D92A938B1077B
:1000A000E1F70C9460000C94000080E181BB8FE0CC
:1000B00084BBAC9AAD9A8EE28ABBD99ADD9A089538
:1000C0001F931092B3011092AF011092B401A0E0FF
:1000D000B0E00E945B15802D992780938701A1E0F5
:1000E000B0E00E945B15802D992780930001A2E06B
:1000F000B0E00E945B15802D9927809388010E94B3
:100100003D110E9455000E940C02809187018130B0
:1001100019F40E94FF0A02C00E94EF0A7894A89A7C
:100120000E94E9010E94BE060E94C6060E94870E38
:100130000E94E3060E942107809182018130C1F470
:10014000109282018091B301882361F40E94BB0B5D
:1001500080919301882321F080910201823014F074
:100160000E94830C0E94F80B0E94FD0B0E94190F45
:10017000809186019091B301813041F4992331F44B
:100180000E947F0A0E942A0E0E94860D809185019E
:10019000813059F58091B301882339F5AA9A0E94DC
:1001A0000F0A80919301882359F40E9490050E94C0
:1001B000F6040E94E5050E9472070E94970814C089
:1001C00080910201823044F00E94E5050E9472078E
:1001D0000E9497080E94550780910201833024F005
:1001E0000E9490050E94F604AA98809180018130B7
:1001F00081F58091B301882361F51092800180918F
:100200009301882321F080910201833014F00E9431
:100210002107809190019091910101969093910115
:10022000809390018091900190919101CC9769F415
:1002300080918E0190918F01019690938F01809310
:100240008E0110929101109290010E945B090E9410
:10025000D60610918101113009F06ECF8091B30163
:10026000882309F069CF109281018091A401813027
:1002700019F0823059F406C00E946D0782E0809325
:10028000A40104C00E9450071093A401809193011F
:10029000813009F051CF8091B301882309F04CCF10
:1002A00080919201813009F047CF109292018091A4
:1002B0000201813071F082301CF4882339F03CCF88
:1002C000823061F0833009F037CF15C00E946D078E
:1002D00033CF0E9450070E948B022ECF0E945007FE
:1002E00064E084E00E9486010E94BE060E94C60669
:1002F0000E94E30621CF0E94500764E084E00E9440
:1003000086010E94BE060E94C60612CF482FD998C9
:1003100027E030E0DB98000000000000000081E0F2
:1003200090E0022E02C0880F991F0A94E2F78423FE
:1003300011F0DA9A01C0DA98000000000000000015
:10034000DB9A0000000000000000215030408FEFD9
:100350002F3F3807F9F627E030E0DB980000000077
:100360000000000081E090E0022E02C0880F991F7B
:100370000A94E2F7862311F0DA9A01C0DA980000B5
:10038000000000000000DB9A0000000000000000F8
:10039000215030408FEF2F3F3807F9F6DB98DA987D
:1003A000D99A089564E084E00E9486016CE480E0BC
:1003B0000E94860110928201809182018823E1F3DC
:1003C0006AE08CE60E94860160E085E00E9486017A
:1003D00008950E94D20110928001809180018823AB
:1003E000E1F30E94CE060E948B0210928001809160
:1003F00080018823E1F3109280018091800188239D
:10040000E1F31092800164E084E00E9486016CE4D4
:1004100080E00E948601089582E083BF82E48EBD61
:100420008AE189BF86E087BD80EF82BD83E4809347
:100430008A0080E280937D0008951F920F920FB68C
:100440000F9211248F939F93809184018F5F8093EB
:10045000840180918401883439F591E0909383017F
:1004600010928401809181038F5F8093810380913A
:100470008103843631F4109281039093800190932C
:10048000810180918103823311F4909381018091E5
:1004900080038F5F80938003809180038A3021F4F2
:1004A00010928003909382019F918F910F900FBEC5
:1004B0000F901F901895282F80538A3010F090E0ED
:1004C00005C0203311F49AE001C0982F822F815487
:1004D0008A3110F4922F9653822F81568A3110F46C
:1004E000922F9C532D3211F499E403C02E3209F45B
:1004F00091E4892F992787FD909508958D3211F405
:1005000089E405C0803311F48AE001C08053992743
:1005100087FD9095089560E085E00E94860163E87C
:1005200086E00E94860160E987E00E94860160E023
:1005300085E00E94860164E886E00E94860161E908
:1005400087E00E94860160E085E00E94860165E800
:1005500086E00E94860162E987E00E94860160E0F1
:1005600085E00E94860166E886E00E94860163E9D4
:1005700087E00E94860160E085E00E94860167E8CE
:1005800086E00E94860164E987E00E94860160E0BF
:1005900085E00E94860168E886E00E94860165E9A0
:1005A00087E00E94860160E085E00E94860169E89C
:1005B00086E00E94860166E987E00E94860160E08D
:1005C00085E00E9486016AE886E00E94860167E96C
:1005D00087E00E94860160E085E00E94860161EA72
:1005E00086E00E94860168E987E00E94860160E05B
:1005F00085E00E94860162EA86E00E94860169E940
:1006000087E00E94860160E085E00E94860163EA3F
:1006100086E00E9486016AE987E00E94860160E028
:1006200085E00E94860164EA86E00E9486016BE90B
:1006300087E00E94860160E085E00E94860165EA0D
:1006400086E00E9486016CE987E00E94860160E0F6
:1006500085E00E94860166EA86E00E9486016DE9D7
:1006600087E00E94860160E085E00E94860167EADB
:1006700086E00E9486016EE987E00E94860160E0C4
:1006800085E00E94860168EA86E00E9486016FE9A3
:1006900087E00E94860160E085E00E9486016FEBA2
:1006A00086E00E94860160EA87E00E94860160E0A1
:1006B00085E00E94860160EC86E00E94860161EA86
:1006C00087E00E94860160E085E00E94860161EC7F
:1006D00086E00E94860162EA87E00E94860160E06F
:1006E00085E00E94860162EC86E00E94860163EA52
:1006F00087E00E94860160E085E00E94860163EC4D
:1007000086E00E94860164EA87E00E94860160E03C
:1007100085E00E94860164EC86E00E94860165EA1D
:1007200087E00E94860160E085E00E94860165EC1A
:1007300086E00E94860166EA87E00E94860160E00A
:1007400085E00E94860166EC86E00E94860167EAE9
:1007500087E00E94860160E085E00E9486016DEDE1
:1007600086E00E94860168EA87E00E94860160E0D8
:1007700085E00E9486016EED86E00E94860169EAAE
:1007800087E00E94860160E085E00E9486016FEDAF
:1007900086E00E9486016AEA87E00E94860160E0A6
:1007A00085E00E94860160EE86E00E9486016BEA89
:1007B00087E00E94860160E085E00E94860161EE8C
:1007C00086E00E9486016CEA87E00E94860160E074
:1007D00085E00E94860162EE86E00E9486016DEA55
:1007E00087E00E94860160E085E00E94860163EE5A
:1007F00086E00E9486016EEA87E00E94860160E042
:1008000085E00E94860164EE86E00E9486016FEA20
:1008100087E00E94860160E085E00E9486016BEF20
:1008200086E00E94860160EB87E00E94860160E01E
:1008300085E00E9486016CEF86E00E94860161EBF4
:1008400087E00E94860160E085E00E9486016DEFEE
:1008500086E00E94860162EB87E00E94860160E0EC
:1008600085E00E9486016EEF86E00E94860163EBC0
:1008700087E00E94860160E085E00E9486016FEFBC
:1008800086E00E94860164EB87E00E94860161E0B9
:1008900085E00E94860160E086E00E94860165EBAB
:1008A00087E00E94860161E085E00E94860161E0A8
:1008B00086E00E94860166EB87E00E94860108952B
:1008C000CF92DF92EF92FF920F931F93CF93DF931C
:1008D0006C01062FEC0115C06D2F772785E00E9473
:1008E00086016C2F86E00E948601F701EE0FFF1F44
:1008F000EE0DFF1DE05EFE4F608187E00E948601E5
:100900002196C6010996E02EFF24C817D90720F3C7
:1009100086010C5F1F4F612F772785E00E948601BB
:10092000602F86E00E948601E701CC0FDD1FCE0D0F
:10093000DF1DC05EDE4F698187E00E9486018A81EB
:10094000882381F086010E5D1F4F612F772785E098
:100950000E948601602F86E00E9486016A8187E0FE
:100960000E948601DF91CF911F910F91FF90EF9030
:10097000DF90CF9008950F931F93CF93DF938C0157
:10098000EC010EC06D2F772785E00E9486016C2F49
:1009900086E00E94860160E087E00E948601219641
:1009A000C8010996C817D90768F38091A201992751
:1009B000FC01EE0FFF1FE80FF91FE05EFE4F828182
:1009C000882379F00E5D1F4F612F772785E00E9405
:1009D0008601602F86E00E94860160E087E00E9429
:1009E0008601DF91CF911F910F9108951F93CF93AF
:1009F000DF9380913C0390913D0366E170E00E949B
:100A000011159B0177FD1BC0CB016AE070E00E94CD
:100A10001115182F1695C9016AE070E00E94111592
:100A200087E090E0861B91092EE130E0829FE00193
:100A3000839FD00D929FD00D11242A9616C0309519
:100A400021953F4FC9016AE070E00E941115182FEF
:100A500016951C5FC9016AE070E00E9411158EE1D5
:100A6000689FE0011124C650DF4F80911C019091D6
:100A70001D01C817D90739F080911C0190911D0103
:100A80000E94BB0404C08091A201811721F0612F54
:100A9000CE010E9460041093A201D0931D01C09367
:100AA0001C01DF91CF911F9108950F931F93CF9356
:100AB000DF93EC01062F10E06D2F772785E00E9471
:100AC00086016C2F86E00E948601E02FFF27E25C02
:100AD000FE4F608187E00E9486016E96125E103F95
:100AE00059F7DF91CF911F910F9108951F93CF93E5
:100AF000DF93EC0110E06D2F772785E00E948601DF
:100B00006C2F86E00E94860160E087E00E948601EB
:100B10006E96125E103F79F7DF91CF911F91089585
:100B20001F93CF93DF9380913E0390913F0366E143
:100B300070E00E9411159B012A5F3F4F37FD12C0E4
:100B4000C9016AE070E00E941115182F16951C5F0C
:100B5000C9016AE070E00E941115C6E8D0E0C61B2A
:100B6000D10913C0309521953F4FC9016AE070E06B
:100B70000E941115182F1695C9016AE070E00E94B5
:100B80001115C62FDD27C957DF4F80911E019091A7
:100B90001F01C817D90739F080911E0190911F01DC
:100BA0000E94760504C08091A301811721F0612F76
:100BB000CE010E9455051093A301D0931F01C0934D
:100BC0001E01DF91CF911F910895FF920F931F9304
:100BD000CF93DF9380914E0390914F038E559040B9
:100BE00063E070E00E941115EB016A3071051CF0A2
:100BF000C9E0D0E004C077FF02C0C0E0D0E080913F
:100C00008C0190918D01C817D90709F47DC0C230BD
:100C1000D10514F468E101C068E084E00E94860117
:100C2000D0938D01C0938C01C530D105B9F1C63088
:100C3000D1057CF4C230D10521F1C330D1051CF4BB
:100C40002197A9F419C0C330D10501F1249779F493
:100C500021C0C730D10549F1C730D1051CF1C830DA
:100C6000D10531F1299719F45BE8F52E23C048E846
:100C7000F42E04E810E820C038E8F32E04E811E868
:100C80001BC028E8F22E04E812E816C098E8F92EF6
:100C900004E811C088E8F82E05E80DC008E8F02E39
:100CA00006E809C018E8F12E05C0B9E8FB2E02C01D
:100CB000AAE8FA2E07E813E860E085E00E948601C2
:100CC00060E286E00E948601612F87E00E94860133
:100CD00060E085E00E9486016EE386E00E94860166
:100CE000602F87E00E94860160E085E00E94860117
:100CF0006CE586E00E9486016F2D87E00E948601E8
:100D000060E084E00E948601DF91CF911F910F91F6
:100D1000FF900895EF92FF920F931F93CF93DF936D
:100D20007A019EE1699FB0011124680F711D8B014A
:100D3000020F111D10928203EB0116C06D2F772751
:100D400085E00E9486016C2F86E00E9486018091DA
:100D50008203F701E80FF11D60818F5F80938203AA
:100D600087E00E9486012196C017D10738F3DF91F2
:100D7000CF911F910F91FF90EF90089524E043E0F1
:100D800051E06EE088E10E948A06089525E047E080
:100D900051E06EE082E00E948A06089520E14CE076
:100DA00051E062E087E00E948A0608958091880100
:100DB000813041F42091B50146EB51E061E08AE0D9
:100DC0000E948A06089560E085E00E94860160E244
:100DD00086E00E94860160E887E00E94860160E06C
:100DE00085E00E9486016EE386E00E94860164E849
:100DF00087E00E94860160E085E00E9486016CE544
:100E000086E00E94860168E887E00E9486010895D6
:100E100060E085E00E9486016FEC86E00E9486011A
:100E20006CE887E00E94860161E085E00E9486010F
:100E30006BE086E00E9486016DE887E00E948601F3
:100E4000089589ED8093820360E085E00E94860129
:100E50006091820386E00E94860164E587E00E943B
:100E60008601809182038F5F809382038C3D60F3C3
:100E700085EE8093820360E085E00E9486016091A8
:100E8000820386E00E94860164E587E00E94860175
:100E9000809182038F5F80938203883E60F3089580
:100EA0006CE480E00E948601089580915003909147
:100EB0005103843B910544F48091A401882361F49B
:100EC00081E08093A40108958091A401181614F480
:100ED0000E9450071092A401089562E480E00E94ED
:100EE00086010895EF92FF920F931F93CF93DF93A4
:100EF000CDB7DEB72D970FB6F894DEBF0FBECDBFCE
:100F0000DE011196E8E4F1E083E001900D9281505A
:100F1000E1F780914603909147036EE170E00E94F3
:100F200011158E01075F1F4FCB0177FF02C080E0D4
:100F300090E04AE050E0B8010E94CC14F801019022
:100F40000020E9F73197EE2EE01A10928203FF2479
:100F50000AC00E0F1F1FEC0FFD1F81850E945B0250
:100F6000F8018083F394EF2DFF278E2D992787FDBD
:100F700090958E010C5F1F4FE817F90754F3F0921C
:100F8000820323E0AE014F5F5F4F6EE088E10E9475
:100F90008A062E2DA8016EE08BE18E190E948A062A
:100FA0002D960FB6F894DEBF0FBECDBFDF91CF9167
:100FB0001F910F91FF90EF900895EF92FF920F9382
:100FC0001F93CF93DF93CDB7DEB72F970FB6F8946B
:100FD000DEBF0FBECDBF85E0FE01369611928A9529
:100FE000E9F780919C0190919D018E01055F1F4F53
:100FF0004AE050E0B8010E94CC14F80101900020B2
:10100000E9F73197EE2EE01A10928203FF240AC00E
:101010000E0F1F1FEC0FFD1F83850E945B02F8015E
:101020008083F394EF2DFF278E2D992787FD9095D0
:101030008E010F5F1F4FE817F90754F3F0928203F8
:1010400024E0AE014A5F5F4F67E089E10E948A06B3
:101050002E2DA80167E08CE18E190E948A068091EE
:101060009C0190919D0118161906C4F460E085E07A
:101070000E9486016FEC86E00E9486016CE887E0A2
:101080000E94860161E085E00E9486016BE086E0B7
:101090000E94860160E087E00E94860180919C01A9
:1010A00090919D0197FF18C060E085E00E94860145
:1010B0006FEC86E00E94860160E087E00E94860176
:1010C00061E085E00E9486016BE086E00E94860177
:1010D0006DE887E00E94860180919C0190919D01BE
:1010E000892BC1F460E085E00E9486016FEC86E008
:1010F0000E94860160E087E00E94860161E085E051
:101100000E9486016BE086E00E94860160E087E035
:101110000E9486012F960FB6F894DEBF0FBECDBF9A
:10112000DF91CF911F910F91FF90EF900895EF9273
:10113000FF920F931F93CF93DF93CDB7DEB72B971B
:101140000FB6F894DEBF0FBECDBFDE011196EBE403
:10115000F1E083E001900D928150E1F78E01085F8C
:101160001F4F4AE050E0B80180914C0390914D032D
:101170000E94CC14F80101900020E9F73197EE2E7F
:10118000E01A10928203FF240AC00E0F1F1FEC0FFB
:10119000FD1F80850E945B02F8018083F394EF2D90
:1011A000FF278E2D992787FD90958E010C5F1F4F8D
:1011B000E817F90754F3F092820323E0AE014F5F82
:1011C0005F4F6EE08DE00E948A062E2DA8016EE032
:1011D00080E18E190E948A062B960FB6F894DEBF26
:1011E0000FBECDBFDF91CF911F910F91FF90EF9078
:1011F0000895EF92FF920F931F93CF93DF93CDB794
:10120000DEB72B970FB6F894DEBF0FBECDBFDE0161
:101210001196EEE4F1E083E001900D928150E1F748
:101220008E01085F1F4F4AE050E0B80180915203E1
:10123000909153030E94CC14F80101900020E9F72B
:101240003197EE2EE01A10928203FF240AC00E0F8F
:101250001F1FEC0FFD1F80850E945B02F801808339
:10126000F394EF2DFF278E2D992787FD90958E0102
:101270000C5F1F4FE817F90754F3F092820323E045
:10128000AE014F5F5F4F6DE08DE00E948A062E2D0C
:10129000A8016DE080E18E190E948A062B960FB698
:1012A000F894DEBF0FBECDBFDF91CF911F910F919C
:1012B000FF90EF900895EF92FF920F931F93CF93BB
:1012C000DF93CDB7DEB728970FB6F894DEBF0FBE19
:1012D000CDBF19828AE08A8380918E0190918F011F
:1012E0008E010A5F1F4F4AE050E0B8010E94CC1403
:1012F000F80101900020E9F73197EE2EE01A1092E4
:101300008203FF240DC08E010D5F1F4F0E0F1F1FA4
:10131000EC0FFD1F86810E945B02F8018083F3942D
:10132000EF2DFF278E2D992787FD9095E817F90758
:1013300054F3F092820380918E0190918F018E017F
:101340000D5F1F4F0A976CF421E0AE014F5F5F4FB6
:101350006EE082E00E948A0621E0A8016EE083E050
:1013600004C022E0A8016EE082E00E948A0680911B
:101370009001909191018E010A5F1F4F4AE050E069
:10138000B8010E94CC14F80101900020E9F73197D0
:10139000EE2EE01A10928203FF240DC08E010D5F25
:1013A0001F4F0E0F1F1FEC0FFD1F86810E945B0257
:1013B000F8018083F394EF2DFF278E2D992787FD69
:1013C0009095E817F90754F3F09282038091900109
:1013D000909191018E010D5F1F4F0A976CF421E0EF
:1013E000AE014E5F5F4F6EE085E00E948A0621E00D
:1013F000A8016EE086E004C022E0A8016EE085E06E
:101400000E948A0628960FB6F894DEBF0FBECDBFA5
:10141000DF91CF911F910F91FF90EF9008950F935F
:101420001F938091A602843409F064C060E070E0EC
:10143000A7EAB2E08C91FD0121811281038114960B
:101440006134710509F456C0422F55274D53504061
:10145000E0915101F0915201E60FF71F9927CD97C6
:10146000880F991F880F991F9A01689413F8359572
:1014700027951694E1F7822B932B808360347105B6
:10148000C9F1212F33272D533040FB013196809134
:10149000510190915201E80FF91F4F70507084E094
:1014A000440F551F8A95E1F7C90195958795959544
:1014B0008795482B592B40836F337105D9F0FB0179
:1014C00032968091510190915201E80FF91F2370DB
:1014D000307086E0220F331F8A95E1F7802F99271D
:1014E000CD97282B392B20836E33710519F06D5F52
:1014F0007F4FA0CF109285011F910F9108950F93F8
:101500001F938091CC01843409F064C060E070E0E6
:10151000ADECB1E08C91FD01218112810381149623
:101520006134710509F456C0422F55274D53504080
:10153000E0915301F0915401E60FF71F9927CD97E1
:10154000880F991F880F991F9A01689413F8359591
:1015500027951694E1F7822B932B808360347105D5
:10156000C9F1212F33272D533040FB013196809153
:10157000530190915401E80FF91F4F70507084E0AF
:10158000440F551F8A95E1F7C90195958795959563
:101590008795482B592B40836F337105D9F0FB0198
:1015A00032968091530190915401E80FF91F2370F6
:1015B000307046E0220F331F4A95E1F7802F9927BC
:1015C000CD97282B392B20836E33710519F06D5F71
:1015D0007F4FA0CF109286011F910F91089582E254
:1015E00089B910BC80B91CBE909A28E92AB996E83E
:1015F00090BD82EC8BB921B99CBF82B9089582E27B
:1016000089B910BC80B91CBE909A88E98AB926E8CD
:1016100020BD92EC9BB980E981B92CBF92B90895A5
:10162000159BFECF83B908951F920F920FB60F92AC
:1016300011248F939F93EF93FF939CB19093830317
:101640009D3081F48091A601813061F4AB981092B5
:10165000A60180938601E0917F03FF27E653FE4FAA
:1016600090832CC08091A601882319F0813031F538
:1016700013C0933239F480918601882319F481E0F4
:101680008093A60110927F0380917F03E82FFF27AC
:10169000E653FE4F90830CC0E0917F03FF27E65393
:1016A000FE4F908380917F03853930F480917F03D2
:1016B0008F5F80937F0302C01092A601FF91EF918C
:1016C0009F918F910F900FBE0F901F9018951F92B2
:1016D0000F920FB60F9211248F939F93EF93FF9366
:1016E00093B1909384039D3081F48091A501813062
:1016F00061F4AB981092A50180938501E0917C0381
:10170000FF27EC55FD4F90832DC08091A5018823C4
:1017100019F0813039F514C0933241F4809185017C
:10172000882321F481E08093A501AB9A10927C0379
:1017300080917C03E82FFF27EC55FD4F90830CC070
:10174000E0917C03FF27EC55FD4F908380917C0353
:10175000853930F480917C038F5F80937C0302C0D5
:101760001092A501FF91EF919F918F910F900FBE65
:101770000F901F901895CF93DF93CDB7DEB72A97C0
:101780000FB6F894DEBF0FBECDBF83E289831A8205
:1017900083E68B831C821D8286E890E060E070E126
:1017A0000E9411159C0160E470E00E941115635CB9
:1017B0006E83C90160E470E00E941115835C8F8321
:1017C0008DE08887FE0131969E01275F3F4F808123
:1017D000159BFECF83B93196E217F307C1F72A961E
:1017E0000FB6F894DEBF0FBECDBFDF91CF91089545
:1017F00085B392E0892785BB089590918B01913044
:1018000019F485B3892785BB08951F920F920FB6EF
:101810000F9211242F933F935F936F937F938F9336
:101820009F93AF93BF938091A7019091A801892BBB
:1018300081F484B595B59093AE018093AD018EB5DA
:101840008F7B8EBD81E090E09093A8018093A701EB
:1018500041C084B595B59093AC018093AB012EB592
:1018600020642EBD2091AD013091AE01821B930BFF
:101870001092A8011092A701865698406CE271E080
:101880000E94FD147093AA016093A90177FF05C01F
:101890001092AA011092A90109C06730710534F0B5
:1018A00086E090E09093AA018093A9012091A9017C
:1018B0003091AA0180910201992787FD9095281700
:1018C000390741F0263031052CF42093020181E0E4
:1018D00080939201BF91AF919F918F917F916F9172
:1018E0005F913F912F910F900FBE0F901F90189511
:1018F0001F920F920FB60F92112413BC0F900FBEC0
:101900000F901F90189580914603909147039093F4
:10191000950180939401809194019091950120917B
:10192000960130919701821B930B909399018093BC
:1019300098018091940190919501909397018093E3
:10194000960180919A0190919B012091980130918C
:101950009901820F931F90939B0180939A0180912C
:101960009E018430F1F410929E0160919A01709171
:101970009B01882777FD8095982F0E94521220E0C6
:1019800030E040EC5FE30E9498110E94BB1270931C
:101990009D0160939C0110929B0110929A010E94FC
:1019A000DD0780919E018F5F80939E010895BF9215
:1019B000CF92DF92EF92FF920F931F93CF93DF931B
:1019C000CDB7DEB760970FB6F894DEBF0FBECDBFC0
:1019D00019821A821B821C8280919802909199022E
:1019E000909388038093870380919A0290919B0241
:1019F0009093860380938503809187039091880359
:101A00008E01055F1F4F4AE050E0B8010E94CC14E0
:101A1000F80101900020E9F73197BE2EB01ACC24CE
:101A2000DD240DC0EC0CFD1CF70180810E945B02DF
:101A30000C0D1D1DF80180830894C11CD11C8B2D39
:101A4000992787FD90952BE0E22EF12CEC0EFD1EE0
:101A50008E010B5F1F4FC816D90624F324E0AE0198
:101A60004F5F5F4F61E08CE00E948A062B2DA8013A
:101A700061E080E18B190E948A0680918503909134
:101A800086034AE050E0B7010E94CC14F7010190B0
:101A90000020E9F73197DE2EDE18EE24FF240DC07A
:101AA000FE01EE0DFF1D83850E945B020E0D1F1DC2
:101AB000F80180830894E11CF11C8D2D992787FD86
:101AC00090958E010B5F1F4FE816F9064CF324E04A
:101AD000AE014F5F5F4F62E08CE00E948A062D2DC1
:101AE000A80162E080E18D190E948A0660960FB617
:101AF000F894DEBF0FBECDBFDF91CF911F910F9144
:101B0000FF90EF90DF90CF90BF9008958F929F92BB
:101B1000BF92CF92DF92EF92FF920F931F93CF93DA
:101B2000DF93CDB7DEB760970FB6F894DEBF0FBE78
:101B3000CDBF19821A821B821C8280906003909014
:101B400061038E01055F1F4F4AE050E0B8018091AC
:101B50005E0390915F030E94CC14F8010190002075
:101B6000E9F73197BE2EB01ACC24DD240DC0EC0C61
:101B7000FD1CF70180810E945B020C0D1D1DF80108
:101B800080830894C11CD11C8B2D992787FD9095CB
:101B90003BE0E32EF12CEC0EFD1E8E010B5F1F4F80
:101BA000C816D90624F324E0AE014F5F5F4F64E00E
:101BB0008CE00E948A062B2DA80164E080E18B193D
:101BC0000E948A064AE050E0B701C4010E94CC148A
:101BD000F70101900020E9F73197DE2EDE18EE24A0
:101BE000FF240DC0FE01EE0DFF1D83850E945B02E8
:101BF0000E0D1F1DF80180830894E11CF11C8D2D32
:101C0000992787FD90958E010B5F1F4FE816F90607
:101C10004CF324E0AE014F5F5F4F65E08CE00E9423
:101C20008A062D2DA80165E080E18D190E948A06A3
:101C300060960FB6F894DEBF0FBECDBFDF91CF9197
:101C40001F910F91FF90EF90DF90CF90BF909F90EA
:101C50008F900895DF92EF92FF920F931F93CF938F
:101C6000DF93CDB7DEB72C970FB6F894DEBF0FBE6B
:101C7000CDBF1D821E821F8218868E01075F1F4FF7
:101C80004AE050E0B8018091A0029091A1020E9428
:101C9000CC14F80101900020E9F73197DE2ED01A1C
:101CA000EE24FF240DC0FE01EE0DFF1D81850E9474
:101CB0005B020E0D1F1DF80180830894E11CF11CCE
:101CC0008D2D992787FD90958E010F5F1F4FE81688
:101CD000F9064CF323E0AE014B5F5F4F61E088E112
:101CE0000E948A062D2DA80161E08BE18D190E94CA
:101CF0008A062C960FB6F894DEBF0FBECDBFDF91DB
:101D0000CF911F910F91FF90EF90DF90089522E007
:101D100047E551E061E08AE10E948A0608958091DA
:101D20009802909199029093880380938703809101
:101D30009A0290919B0290938603809385038091F1
:101D40008703909188038091850390918603809109
:101D5000870390918803809185039091860308956D
:101D6000F89488E190E028E00FB6F894A89581BD3A
:101D70000FBE21BDFFCF64E084E00E948601209168
:101D8000B50146EB51E062E08AE00E948A0668E015
:101D900084E00E94860126E049E551E065E08AE0A2
:101DA0000E948A0680910001813021F423E041E7FE
:101DB00051E003C023E044E751E065E081E10E9487
:101DC0008A0660E084E00E94860126E04FE551E04B
:101DD00066E08AE00E948A0680918701813021F4C2
:101DE00023E041E751E003C023E044E751E066E02F
:101DF00081E10E948A0626E045E651E067E08AE03C
:101E00000E948A0680918801813021F423E041E715
:101E100051E003C023E044E751E067E081E10E9424
:101E20008A0626E04BE651E068E08AE00E948A06D6
:101E300008959D998EC08091AF018F5F8093AF010F
:101E400091E09093B1018091AF01853009F085C098
:101E50008091B301882339F49093B3011092B401B7
:101E60000E94BB0E78C09091B401913071F58091C1
:101E70008701882319F49093870102C0109287018B
:101E800080918701A0E0B0E0082E0E94631568E011
:101E900084E00E94860126E04FE551E066E08AE09A
:101EA0000E948A0680918701813021F423E041E776
:101EB00051E003C023E044E751E066E081E10E9485
:101EC0008A0660E084E00E9486018091B40182303D
:101ED00079F580918801882321F481E0809388013D
:101EE00002C01092880180918801A2E0B0E0082E23
:101EF0000E94631568E084E00E94860126E045E6C2
:101F000051E067E08AE00E948A0680918801813072
:101F100021F423E041E751E003C023E044E751E02E
:101F200067E081E10E948A0660E084E00E94860109
:101F30008091B401833089F41092B301F89488E160
:101F400090E028E00FB6F894A89581BD0FBE21BDA2
:101F5000FFCF1092AF011092B1019C997FC1909177
:101F6000B301913009F080C19093B2018091B0012A
:101F70008F5F8093B0018091B001853009F074C10A
:101F80001092B0018091B401813009F44CC08130CD
:101F900038F0823009F4A1C0833009F065C1FEC079
:101FA0009093B40164E084E00E9486012091B50121
:101FB00046EB51E062E08AE00E948A0626E049E5AD
:101FC00051E065E08AE00E948A068091000181303C
:101FD00021F423E041E751E003C023E044E751E06E
:101FE00065E081E10E948A0668E084E00E94860143
:101FF00026E04FE551E066E08AE00E948A06809183
:102000008701813021F423E041E751E003C023E060
:1020100044E751E066E081E10E948A0660E084E0E6
:102020000E948601FDC082E08093B40164E084E0F8
:102030000E9486012091B50146EB51E062E08AE002
:102040000E948A0626E049E551E065E08AE00E94A8
:102050008A0680910001813021F423E041E751E0BC
:1020600003C023E044E751E065E081E10E948A0675
:1020700026E04FE551E066E08AE00E948A06809102
:102080008701813021F423E041E751E003C023E0E0
:1020900044E751E066E081E10E948A0668E084E05E
:1020A0000E94860126E045E651E067E08AE00E9452
:1020B0008A0680918801813021F423E041E751E0D4
:1020C00003C023E044E751E067E081E10E948A0613
:1020D00060E084E00E948601B9C083E08093B4018F
:1020E00064E084E00E9486012091B50146EB51E056
:1020F00062E08AE00E948A0626E049E551E065E058
:102100008AE00E948A0680910001813021F423E058
:1021100041E751E003C023E044E751E065E081E19D
:102120000E948A0626E04FE551E066E08AE00E94C0
:102130008A0680918701813021F423E041E751E054
:1021400003C023E044E751E066E081E10E948A0693
:1021500026E045E651E067E08AE00E948A06809129
:102160008801813021F423E041E751E003C023E0FE
:1021700044E751E067E081E10E948A0668E084E07C
:102180000E94860126E04BE651E068E08AE00E946A
:102190008A0660E084E00E94860108951092B401EE
:1021A00064E084E00E9486012091B50146EB51E095
:1021B00062E08AE00E948A0668E084E00E9486016C
:1021C00026E049E551E065E08AE00E948A068091B8
:1021D0000001813021F423E041E751E003C023E016
:1021E00044E751E065E081E10E948A0660E084E016
:1021F0000E94860126E04FE551E066E08AE00E94F9
:102200008A0680918701813021F423E041E751E083
:1022100003C023E044E751E066E081E10E948A06C2
:1022200026E045E651E067E08AE00E948A06809158
:102230008801813021F423E041E751E003C023E02D
:1022400044E751E067E081E10E948A0626E04BE620
:1022500051E068E08AE00E948A0608951092B00179
:102260008091B1018091B2010895813029F4A0E0FC
:10227000B0E0062E0E9463150895EF92FF920F932F
:102280001F93CF93DF93CDB7DEB764970FB6F89463
:10229000DEBF0FBECDBF40E050E08E010F5F1F4F8D
:1022A000842F9927DC01AD5FBF4F0E945B15202D65
:1022B0003327F801E80FF91F20832223F1F04F5F45
:1022C0005F4F2F3F69F7108218C0FE01E00FF11F2A
:1022D00081810E945B020A541E4FF80180830E2DFB
:1022E00011278091B5010894E11CF11C992787FD05
:1022F0009095081719074CF30EC0DE011196FD01E9
:1023000001900020E9F73197EA1BFB0BE093B50140
:10231000EE24FF24E4CF64960FB6F894DEBF0FBE20
:10232000CDBFDF91CF911F910F91FF90EF90089556
:10233000A8E1B0E0EEE9F1E10C942A1569837A8313
:102340008B839C832D833E834F835887B1E18B2EF3
:10235000912C8C0E9D1EB401CE0101960E942D146D
:102360008E01075F1F4FB801CE0105960E942D1404
:102370002989223008F46AC03985323008F468C0EF
:102380008A899A8589278A8B243009F463C0223090
:1023900009F460C0343041F41D8A1E8A1F8A188EE9
:1023A0001C8A1B8AB40177C0323009F458C06B898B
:1023B0007C898B859C85681B790B7C8B6B8B2D892D
:1023C0003E894F89588DED84FE840F8518892E151E
:1023D0003F054007510740F4220F331F441F551F8C
:1023E000615070407C8B6B8B80E090E0A0E0B0E4AB
:1023F000AA24BB24650160E070E02E153F0540076C
:10240000510740F0A82AB92ACA2ADB2A2E193F0907
:10241000400B510BB695A79597958795220F331FC3
:10242000441F551F6F5F7F4F6F31710531F7D60124
:10243000C5018F779070A070B07080349105A105B0
:10244000B10589F0AD8ABE8ACF8AD88EB40123C087
:10245000B80121C03217D1F767E771E01CC084E0F2
:10246000898BB40118C0A7FCEDCF211531054105BA
:10247000510541F380E490E0A0E0B0E0A80EB91E61
:10248000CA1EDB1E80E89FEFAFEFBFEFA822B92284
:10249000CA22DB22D7CFCB010E940B13ECE0689657
:1024A0000C944615A8E0B0E0E8E5F2E10C94331591
:1024B0009B01AC0183E089831A8257FD51C021152D
:1024C00031054105510539F482E08983CE01019639
:1024D0000E940B134CC0EEE1F0E0FC83EB838A8199
:1024E0008823C9F1203010E0310710E0410710E8DF
:1024F0005107C9F188279927DC01821B930BA40B94
:10250000B50B8D839E83AF83B8872D813E814F812C
:102510005885203080E0380780E0480780E458077D
:10252000A8F6EB81FC81DA01C901880F991FAA1F67
:10253000BB1F31979C01AD01803010E0910710E086
:10254000A10710E4B10778F3FC83EB838D839E83AE
:10255000AF83B887BBCF2D833E834F835887D5CFBA
:1025600081E08A83ACCF60E070E080E09FECE3E044
:1025700028960C944F15ACE0B0E0E1ECF2E10C943D
:10258000341569837A838B839C83BE016B5F7F4F95
:10259000CE0101960E942D148D81823061F082302F
:1025A00050F0843069F48E81882359F52FEF3FEF86
:1025B0004FEF5FE72AC020E030E040E050E025C068
:1025C0002F81388537FDF7CF2F31310564F78EE144
:1025D00090E0821B930B29853A854B855C8504C06E
:1025E00056954795379527958A95D2F78E818823FA
:1025F00061F050954095309521953F4F4F4F5F4F7B
:1026000004C020E030E040E050E8CA01B901E2E057
:102610002C960C9450154F925F926F927F928F92EE
:102620009F92AF92BF92DF92EF92FF920F931F9310
:1026300020E030E040E050E0FC01E480F5800681DD
:102640001781D1808081823038F4D801C701A06120
:10265000AF77B0706FEFD9C0843009F46EC08230AC
:1026600009F471C0E114F1040105110509F46BC00E
:10267000828193816FEF823896070CF06AC062E81E
:102680007FEF681B790B6A3171050CF080C0470140
:102690005801062E04C0B694A794979487940A9480
:1026A000D2F744245524320181E090E0A0E0B0E06C
:1026B00004C0880F991FAA1FBB1F6A95D2F7019704
:1026C000A109B109E822F9220A231B23E114F1042C
:1026D0000105110529F061E0462E512C612C712C69
:1026E00085017401E428F52806291729D801C701B6
:1026F0008F779070A070B07080349105A105B105FE
:1027000009F457C0D801C701CF96A11DB11D60E0E3
:1027100070E08030E0E09E07E0E0AE07E0E4BE0756
:1027200010F061E070E027E0B695A7959795879542
:102730002A95D1F7AF77B07068C080E090E0A0E054
:10274000B0E06FEF62C080E090E0A0E0B0E060E059
:102750005CC0803891058CF7BC0161587F4FD8016F
:10276000C7018F779070A070B07080349105A1057B
:10277000B105A1F08FE390E0A0E0B0E0E80EF91E13
:102780000A1F1B1F17FD28C0D801C701CCCF60E06E
:1027900070E080E090E0A0E0B0E0CCCFE7FEF2CFC8
:1027A00080E490E0A0E0B0E0E80EF91E0A1F1B1FD5
:1027B000E9CFE7FC18C080E090E060E0E61660E05A
:1027C000F60660E0060760E4160710F081E090E08E
:1027D000BC01D801C701A7CF16950795F794E794D8
:1027E0006F5F7F4FD1CFD801C701805C9F4FAF4F44
:1027F000BF4F60E070E08030E0E09E07E0E0AE07B1
:10280000E0E4BE0708F48FCF8CCF282F392F9A2F02
:102810009F77842F8078892B962F97959927979566
:102820008F77482F492B6695852F8078862BD794F4
:10283000DD24D7948F77582F5D29CA01B9011F91E4
:102840000F91FF90EF90DF90BF90AF909F908F908F
:102850007F906F905F904F900895FC01DB01208185
:1028600031819281492F4F7750E0991F9927991F05
:102870008381682F660F692B881F8827881FFD01B9
:102880008183662309F049C02115310541055105B1
:1028900009F470C082E89FEFFD0193838283220FC9
:1028A000331F441F551F220F331F441F551F220F74
:1028B000331F441F551F220F331F441F551F220F64
:1028C000331F441F551F220F331F441F551F220F54
:1028D000331F441F551F83E08C932030F0E03F07E7
:1028E000F0E04F07F0E45F0790F482E89FEF220FDB
:1028F000331F441F551F0197203060E0360760E00A
:10290000460760E4560798F3FD0193838283FD0137
:10291000248335834683578308956F3F71F1862F53
:1029200099278F579040FD019383828383E08C9396
:10293000220F331F441F551F220F331F441F551FE3
:10294000220F331F441F551F220F331F441F551FD3
:10295000220F331F441F551F220F331F441F551FC3
:10296000220F331F441F551F506424833583468331
:102970005783089582E08C93089521153105410510
:10298000510519F484E08C93089544FD02C01C9213
:10299000BECF81E08C93BBCFFB019F01E894423016
:1029A000C4F04532B4F44A3029F497FB1EF49095F4
:1029B00081959F4F642F77270E94FD14805D8A3395
:1029C0000CF0895D8193CB010097A1F716F45DE2CD
:1029D00051931082C9010C94ED14DC01FC010190AB
:1029E0000020E9F73297AE17BF0730F47C91608181
:1029F000708331976D93F7CF0895AA1BBB1B51E1EC
:102A000007C0AA1FBB1FA617B70710F0A61BB70B5E
:102A1000881F991F5A95A9F780959095BC01CD0103
:102A2000089597FB092E07260AD077FD04D0E5DF2D
:102A300006D000201AF4709561957F4F0895F6F73F
:102A4000909581959F4F08952F923F924F925F925C
:102A50006F927F928F929F92AF92BF92CF92DF92AE
:102A6000EF92FF920F931F93CF93DF93CDB7DEB713
:102A7000CA1BDB0B0FB6F894DEBF0FBECDBF0994A7
:102A80002A88398848885F846E847D848C849B84FE
:102A9000AA84B984C884DF80EE80FD800C811B810C
:102AA000AA81B981CE0FD11D0FB6F894DEBF0FBE3B
:102AB000CDBFED010895E199FECFBFBBAEBBE09A5B
:102AC00011960DB20895E199FECFBFBBAEBB0DBA12
:0E2AD00011960FB6F894E29AE19A0FBE08959F
:102ADE0001010200000A3100004400005D5E5F4902
:102AEE005B1D5C00202936410A4107262300230086
:102AFE005464665363655262005161005060005029
:102B0E0060005161005262005363655464666768E9
:102B1E00696A6B6B6A69686700000000000000005C
:102B2E00003A0360020D0A0A1D1A0B160000001A65
:102B3E000D470C1E001529323200000F3C2D3800B7
:102B4E0000191800192A2A000000000000000000D9
:00000001FF
